:020000020000FC
:100000009AC1E1C1189518951895189518951895E5
:1000100018951895F7C01895189518951895119773
:10002000F1F708950F93BF93AF93B3E1A8E8F7DF1B
:100030000A95D9F7AF91BF910F9108950F93CF9380
:10004000DF93CAE00F9304E6EDDFCA95E1F70F9165
:100050000A95B9F7DF91CF910F9108953F065B4F55
:10006000666D7D077F6F777C395E797100010203D1
:100070003909090F0F00A0E6BB27ECE5F0E002C04C
:1000800005910D93E637E1F7B898B998C098C198F3
:100090000895B99A22D00895B99A1FD0B8981DD062
:1000A000B9981BD008955F9358E0B89A16D006957A
:1000B00010F4B99801C0B99A10D0B8980ED05A95DA
:1000C000A1F7B89AB99809D0B89807D0B99BB99A4E
:1000D00004D0B89A02D05F910895B1E0A4EF9FDFF9
:1000E00008955CD0FF93EF93BF93AF93DF93CF93CB
:1000F000E0E7F0E0A4E7B0E054E0E0E7F0E00191F1
:10010000C0E6D0E0C00F08810D935A95C1F7CF919A
:10011000DF91AF91BF91EF91FF91FF93EF93BF9369
:10012000AF93B7DF00E4BFDFB7DFB3DF0091790043
:100130000370006CB8DFE4E7FF2754E06894019196
:100140003EF40F3321F4513011F0002701C0E89440
:10015000541709F40068A7DF5A9589F79DDF99DFE6
:100160000091780000689FDF97DFAF91BF91EF911A
:10017000FF91089542E0DB013090780055E05F93F5
:10018000A0927800AEDF04E64DDF30927800A9DF60
:1001900004E648DF5F915A9591F70895BF93AF93B6
:1001A000E0E7F0E00FEF0395A85EB340E0F70193BE
:1001B0000AE00A95AC59BF4FE0F301930FEF0395A6
:1001C000AA50E8F70193A65FA083AF91BF9108956D
:1001D0000F930AB502600ABD03B7056003BF02E1D1
:1001E00009BD09B7006109BF0F9108950F9300275A
:1001F00000937C0000937D0000937E0000937F00BD
:100200000F910895BFB6FF93EF93DF93CF93E091E3
:100210007C00F0917D00C0917E00D0917F003196EE
:10022000CA1DDA1DE0937C00F0937D00C0937E0030
:10023000D0937F00CF91DF91EF91FF91BFBE1895D2
:10024000E199FECF0F9300E00CBBDFBBCEBB2DBB13
:10025000E29AE19A21960F910895E199FECFDFBBD2
:10026000CEBBE09A2DB321960895112783DF44E099
:10027000DB0137DF1EF4DB0134DFE894B39B09C0F8
:1002800010FFF8CF11FD02C033D001C01D7F1E7FCB
:10029000F1CF10FF2AD011FDEDCFFF93EF93DF9345
:1002A000CF93E0917C00F0917D00C0917E00D091D1
:1002B0007F00EA3FFA05CA05DA0590F012606894FB
:1002C0004A95042F013061F4DD27CC27272F209396
:1002D0007A00B6DF262F20937B00B2DF4BDF089534
:1002E000CF91DF91EF91FF91C5CF11607FDF08952E
:1002F0006894E4E7F0E0E41BFA0900810F5F0A303C
:1003000009F4002700837727E0E7F0E0619101918D
:1003100005D0019103D0019101D00895660F771F98
:10032000A62FB72FAA0FBB1FAA0FBB1F6A0F7B1FD9
:10033000600F7A1D0895AA2499240FE50DBF02E0ED
:100340000EBF00E806BD00E006BD01E0C02E3798F4
:1003500092DEDD27CC2781DF20937A007EDF209399
:100360007B00BA98BB98BC9A33DF78940FEF5ADEC3
:1003700070917A0060917B00B39B78DF02E005BF4B
:1003800000E40BBF42E070917A0060917B00BB27D4
:10039000AA27C49AB39B0ED0A617B707D9F36A153C
:1003A0007A0519F0DB019DDEF5CFC498DB0199DEFB
:1003B000F894FFCF90FE02C0C49A01C0C4980FEF1A
:1003C00031DE90940895BFB6655070406A157A0585
:0C03D0000CF002C077276627BFBE18950E
:00000001FF
